:03200000022100BA
:03202B00022E9BE7
:1021000075BF0143B70843B70453B6F743B6047924
:1021100000780AD9FED8FC785643B602D8FEE5B658
:1021200030E0F475BB9853B70F43B7A053B7FB43E8
:10213000B7027864D8FEE5B730E0DC53B7F775BF77
:102140000078FFE4F6D8FD90F0007F007E06E4F012
:10215000A3DFFCDEFA75819F0221960221DBE49366
:10216000A3F8E493A34003F68001F208DFF480298A
:10217000E493A3F85407240CC8C333C4540F442079
:10218000C8834004F456800146F6DFE4800B010268
:10219000040810204080902A15E47E019360BCA3BF
:1021A000FF543F30E509541FFEE493A360010ECFB6
:1021B00054C025E060A840B8E493A3FAE493A3F8E0
:1021C000E493A3C8C582C8CAC583CAF0A3C8C582A0
:1021D000C8CAC583CADFE9DEE780BE122B48E4F532
:1021E000BF7581C0D280D2B67D02FF12420F7B0143
:1021F0007AF079E6123E7C90F10EEEF0A3EFF01249
:10220000386A122E21124375123B4B80F27C011268
:102210002D8D7F027E002202255FE86480F8E9337D
:10222000E83360110460F0ED33EC337009E8FCE949
:10223000FDEAFEEBFF220460DED3EB9FEA9EE99D00
:10224000E8C2E78CF0C2F795F0400CE8CCF8E9CD95
:10225000F9EACEFAEBCFFB12252A85D0F0580470AC
:102260000320D5B3E80470075002B2D50225699265
:10227000D5EC0460F7E4CCC0E0C398F8603B941858
:102280006008400DD0E0FB022541E4FBFAC9FC8068
:1022900028E830E406E4C9FBE4CAFCE830E305E4DE
:1022A000C9CACBFCE854076010F8C3E913F9EA1374
:1022B000FAEB13FBEC13FCD8F130F52FC3E49CFCD4
:1022C000EF9BFFEE9AFEED99FDD0E0FBEF4E4D4CFB
:1022D000701222DB03022566EC2CFCEF33FFEE3399
:1022E000FEED33FDED30E7EB022541EF2BFFEE3A3B
:1022F000FEED39FDD0E0FB50130BBB000302256956
:10230000ED13FDEE13FEEF13FFEC13FC022541EC81
:102310004D6011E8497017ED33EC3304600DE4FCB7
:10232000FFFEFD22E933E8330470F802255F122531
:102330002A58046009E4CC2481500628500902255B
:1023400069284003022566C0E0EB4A7044B9800664
:10235000D0E0FB022555EF4E701CBD8008EBFFEA74
:10236000FEE9FD80EBE98DF0A4FEE5F00223F8E93B
:10237000CDF9EAFEEBFFEF89F0A4FCE5F0CE89F0A1
:10238000A42EFFE435F0CD89F0A42DFEE435F080D5
:1023900067EF4E7005BD80D780C3EF8BF0A4ACF023
:1023A000EE8BF0A42CFCE435F0F8EF8AF0A42CE5D9
:1023B000F038FCE433CB8DF0A42CFCE5F03BF8EED8
:1023C0008AF0A42CFCE5F038F8E433CF89F0A42C93
:1023D000FCE5F038CF3400CE89F0A42FFFE5F03EC5
:1023E000FEE433C98DF0A42EFEE5F039CD8AF0A4C9
:1023F0002FFFE5F03EFEE43DFD33D0E0FB50070B40
:10240000BB000F022569EC2CFCEF33FFEE33FEED31
:1024100033FD022541022569EC5D046005E859049D
:10242000700302255F12252A580460F6EC4860F21A
:10243000EC7004FDFEFF22C860DB2481C85009C394
:1024400098600250060225669850CAF582E9294B29
:102450004A7005AB8202255575F0007C1A7880C35E
:10246000EF9BEE9AED99400DC3EF9BFFEE9AFEEDC8
:1024700099FDE842F0DC23ACF0D0E0FFD0E0FED0E4
:10248000E0FDAB8220E7101BEB60BAEC2CFCEF33D5
:10249000FFEE33FEED33FD022541E803F830E7059A
:1024A000C0F075F000EF2FFFEE33FEED33FD40B8C6
:1024B00030E7C280AA75F020800E75F01080057597
:1024C000F0087D007E007F003392D530D5031226C0
:1024D000ABEC334010EF33FFEE33FEED33FDEC3366
:1024E000FCD5F0ED22E5F0247EA2D513CC92E7CD09
:1024F000CEFF22EDD2E7CD33EC3392D524814006D6
:10250000E4FFFEFDFC22FCE4CFCECDCC24E0501154
:1025100074FF80EDC3CC13CCCD13CDCE13CECF132F
:10252000CF0470F030D5DE0226ABE9D2E7C933E83C
:1025300033F892D5EDD2E7CD33EC33FC5002B2D56F
:1025400022EC30E7100FBF000C0EBE00080DBD00DE
:10255000040BEB6014A2D5EB13FCED92E7FD2274A3
:10256000FFFCFDFEFF22E480F8A2D574FF13FC7D82
:1025700080E480EFBB010689828A83E0225002E773
:1025800022BBFE02E32289828A83E49322BB010CF0
:10259000E58229F582E5833AF583E0225006E925B4
:1025A00082F8E622BBFE06E92582F8E222E58229CE
:1025B000F582E5833AF583E49322BB010FF8E582C7
:1025C00029F582E5833AF583E028F0225009C58297
:1025D00029F8E58226F622BBFE09C58229F8E22504
:1025E00082F222F8EA2583F583E9932822BB0106CB
:1025F00089828A83F0225002F722BBFE01F322F87F
:10260000BB010DE58229F582E5833AF583E8F022E6
:102610005006E92582C8F622BBFE05E92582C8F2EC
:1026200022BC000BBE0029EF8DF084FFADF022E448
:10263000CCF875F008EF2FFFEE33FEEC33FCEE9D87
:10264000EC984005FCEE9DFE0FD5F0E9E4CEFD22AE
:10265000EDF8F5F0EE8420D21CFEADF075F008EF39
:102660002FFFED33FD4007985006D5F0F222C398B6
:10267000FD0FD5F0EA22A3F8E0C5F025F0F0E582E1
:10268000158270021583E0C838F0E822BB010A8980
:10269000828A83F0E5F0A3F0225006F709A7F0192B
:1026A00022BBFE06F3E5F009F31922C3E49FFFE421
:1026B0009EFEE49DFDE49CFC22EB9FF5F0EA9E4229
:1026C000F0E99D42F0E89C45F022E8600FECC3136E
:1026D000FCED13FDEE13FEEF13FFD8F122E8600FBF
:1026E000EFC333FFEE33FEED33FDEC33FCD8F122C4
:1026F000BB010789828A830229ED5005E9F8022986
:10270000E1BBFE05E9F80229F989828A83022A05DC
:10271000ECF0A3EDF0A3EEF0A3EFF022A882858306
:10272000F0D083D082122733122733122733122797
:1027300033E473E493A3C583C5F0C583C8C582C8D9
:10274000F0A3C583C5F0C583C8C582C822E3F5F0F0
:1027500009E208B5F06BDFF58067E3F5F009E608FC
:10276000B5F05EDFF5805A87F009E608B5F052DF74
:10277000F6804E87F009E208B5F046DFF680428821
:10278000828C8387F009E0A3B5F036DFF6803288CB
:10279000828C8387F009E493A3B5F025DFF58021CF
:1027A00088828C83E3F5F009E0A3B5F014DFF580AF
:1027B0001088828C83E3F5F009E493A3B5F002DF7F
:1027C000F4022878808780E9809080D4803C80154E
:1027D000806C807C809D80B7808D80A3804F8072CC
:1027E000803A02288489828A8363A20188828C834A
:1027F00063A201E493F5F0A363A201E493A363A2AF
:1028000001B5F074DFEDDEEB806E89828A83E4939C
:10281000F5F0A3E208B5F060DFF4805C89828A837A
:10282000E0F5F0A3E608B5F04FDFF5804B89828A2A
:1028300083E0F5F0A3E208B5F03EDFF5803A898247
:102840008A83E493F5F0A3E608B5F02CDFF4802842
:102850008002805389828A8363A20188828C836389
:10286000A201E493F5F0A363A201E0A363A201B582
:10287000F006DFEEDEEC80007FFFB5F0020F2240B5
:10288000027F012289828A8363A20188828C83630A
:10289000A201E0F5F0A363A201E0A363A201B5F0F9
:1028A000D7DFEFDEED80D189828A8363A20188823F
:1028B0008C8363A201E0F5F0A363A201E493A36318
:1028C000A201B5F0B3DFEEDEEC80AD88F0EF600181
:1028D0000E4E60AFED2402B40400509CF582EB2450
:1028E00002B40400509223234582239027C473E747
:1028F00009F608DFFA8046E709F208DFFA803E8829
:10290000828C83E709F0A3DFFA8032E309F608DF5F
:10291000FA8076E309F208DFFA806E88828C83E31E
:1029200009F0A3DFFA806289828A83E0A3F608DFD8
:10293000FA805689828A83E0A3F208DFFA804A800F
:10294000D280FA80C680D4806580F2803180108089
:10295000A680EA809A80A880DA80E280CA803189E5
:10296000828A8363A20188828C8363A201E493A399
:1029700063A201F0A363A201DFF3DEF1800B898281
:102980008A83E493A3F608DFF9ECFAA9F0EDFB22C1
:1029900089828A8363A20188828C8363A201E0A377
:1029A00063A201F0A363A201DFF4DEF280DB89827F
:1029B0008A83E493A3F208DFF980CE88F0EF600108
:1029C0000E4E60C588F0ED2402B4040050BBF582C1
:1029D000EB2402B4040050B1232345822390293F05
:1029E00073E6FC08E6FD08E6FE08E6FF22E0FCA32D
:1029F000E0FDA3E0FEA3E0FF22E2FC08E2FD08E226
:102A0000FE08E2FF22E493FC740193FD740293FE3E
:102A1000740393FF2258F000000000000000000043
:102A200000000000000000000000000000000000A6
:102A300044F0470000000042F03C0000C100C1012A
:102A400042F03A03E848F03E0000000000000000B9
:102A500048F04B000000000000000048F02100009A
:102A600000000000000048F0290000000000000005
:102A70000050F065000000000000000000000000B1
:102A80000000000050F055000000000000000000B1
:102A90000000000000000048F019000000000000E5
:102AA000000048F032000000000000000041F0315A
:102AB0000050F07600000000000000000000000060
:102AC0000000000041F0460041F0180041F07500A0
:102AD000C102C10341F0540041F0530048F0DE0050
:102AE0000000000000000041F110004CF1111F1C1B
:102AF0001F1E1F1E1F1F1E1F1E1F008E198F188CCA
:102B00001C8D1BE4F51DF51EF51FC0D0C0E0C0F004
:102B100043D01812DFF94008D0F0D0E0D0D0D32253
:102B2000D0F0D0E0D0D0C3228F18C0D0C0E0C0F029
:102B300043D01812DFF64008D0F0D0E0D0D0D32236
:102B4000D0F0D0E0D0D0C32275BF0175BA10E4F543
:102B5000BFB19DF18AD111F19C7169F165E4F5B8BD
:102B6000F5B9F5F8F5F9D2AF2275DA0075D97175B6
:102B7000DC01E5DC30E00553D8FE80F675DA00753F
:102B8000D98075DB4975D815E5D820E1FB75D804E7
:102B9000E4F5DBF5DC75D835E5D820E1FBE4F5DBC1
:102BA000F5DC75D835E5D820E1FB75DB4B75DC3AF3
:102BB00075D835E5D820E1FB75DD6075D845E5D8D9
:102BC00020E1FBE4F5DBF5DCF5DD75D871E5D82017
:102BD000E1FB75DA0075D9C075DB4175D815E5D80C
:102BE00020E1FB75B202439002439102E4F5B24347
:102BF0009102F5DA75D9717F02FE7D0812220D7DF2
:102C00000512220D7D0612220D7D0712220D7D096F
:102C100012220D7D0A12220D7D0B12220D7D0C1247
:102C2000220D7D0D7C01B18D75DA0475D92FD10A85
:102C3000B1857F037E007D007CE0B16DB1F8B18786
:102C40007F007E05B176B1EA75D937D101B1877FB2
:102C500001B167B1F8B1877F007E06B176B1EA7540
:102C6000D93FD10AB1857F02B167B1F8B1877F0042
:102C70007E07B176B1EA75D947D101B1877F027E6F
:102C8000007D007CF1B16DB1F8B1877F007E08B1A5
:102C900076B1EA75D94FD101B1877FF07EFF7DFF14
:102CA0007CFFB16DB1F8B1877F007E09B176B1EAE2
:102CB00075D957D101B1877F027E007D007CF4B1C8
:102CC0006DB1F8B1877F007E0AB176B1EA75D95F40
:102CD000D10AB1857F04B167B1F8B1877F007E0B5F
:102CE000B176B1EA75D967D101B1877F03B167B118
:102CF000F8B1877F007E0CB176B1EA75D96FD10A41
:102D0000B1857F017E007D007CF4B16D7FFF7EFF89
:102D10007DFF7C1FB1877F007E0DB1767F007E0036
:102D20007D007C08B14075DA0075D980E4F5D8E5FE
:102D3000D820E1FB53DBBE75D811E5D820E1FB229A
:102D400090F0A412271090F0A7E0F5DB90F0A6E039
:102D5000F5DC90F0A5E0F5DD90F0A4E0F5DE75D8A7
:102D6000F1E5D820E1FB227E007D007CF5B14075C5
:102D7000D8087F007E007D007C00B14075D8087FB8
:102D8000007E007D007C00B14075D80822B14075FE
:102D9000DC01E5DC30E00553D8FE80F62275B20395
:102DA00075800875B2017580FE7586EFE4F5B27521
:102DB000860D75800C75B203F59075B2017590DFC4
:102DC0007591BFF5B275916075B20375B03C75B27F
:102DD0000175B03F75B1FCF5B275B1FC75B201F586
:102DE000C875C908F5B275C908227F007E007D004C
:102DF0007C08B14075DA04227FFF7EFF7DFF7C3FB7
:102E0000227F007E007DA87C0E227F007E007DA0B8
:102E100022F17D75BCDB43BB0443BB03F169F5BF05
:102E20002290F088743FF0C2AFE5D820E1FBC0D912
:102E3000C0DAC0DBC0DCC0DDC0DE75BF80D194E489
:102E4000F5D8E5D820E1FB90F086E5DBF0A3E5DCE2
:102E5000F090F086E030E502716990F086E0FF5472
:102E600007600690F0887438F0D19490F088E05FA5
:102E7000F4F5DB90F087E0F4F5DC75D831E5D82087
:102E8000E1FB75BFC0D0DED0DDD0DCD0DBD0DAD046
:102E9000D9D2AF2275DA0075D98122C0E0C0F0C066
:102EA00083C082C0D075D00063A201C083C082639A
:102EB000A201C000C001C002C003C004C005C0061A
:102EC000C00790F0D3743FF0E5D820E1FBC0D9C033
:102ED000DAC0DBC0DCC0DDC0DE75BF8030C704C235
:102EE000C7F1B7E5B65401604853B6FED19475D822
:102EF00000E5D820E1FBAFDBAEDCEF30E51B30E7CF
:102F00000A90F0547480F0EF547FFFEF30E60A909F
:102F1000F0547440F0EF54BFFFD19490F0D3E05FD1
:102F2000F4F5DBAF06EEF4F5DC75D831E5D820E139
:102F3000FB75BFC0D0DED0DDD0DCD0DBD0DAD0D99D
:102F4000D007D006D005D004D003D002D001D000E5
:102F500063A201D082D08363A201D0D0D082D0837B
:102F6000D0F0D0E03243A82022538FFE75BF017508
:102F7000BBAB22F17D53BBFBF169F5BF2275BF01ED
:102F800075BB9BE4F5BF438F012275C43075C5F84E
:102F900075C23075C3F8E4F5C1D2C22275BF0175A0
:102FA000B41375B50275BF03E4F5BBF5BF43A801C3
:102FB00075880175B3012230002490F03DE004F0E3
:102FC000700690F03CE004F090F03AF1EB90F03DA8
:102FD000E09F90F03CE09E400CC200E48004E4904E
:102FE000F03CF0A3F022EDF090F0A2E0FEA3E0FFB1
:102FF000C3221236B0E5D820E1FBC0D9C0DAC0DB6D
:10300000C0DCC0DDC0DED1F52400B1D3E4F5D8E5E5
:10301000D820E1FB90F0A531A7E5DE1225EDD1F532
:103020002404B1D3E4F5D8E5D820E1FB90F0A53134
:10303000A790000DE5DB1225FF90000CE5DC1225C2
:10304000FF90000BE5DD1225FF90000AE5DE12255A
:10305000FF75D804E4F5D8E5D820E1FB90F0A53160
:10306000A7900011E5DB1225FF900010E5DC12258A
:10307000FF90000FE5DD1225FF90000EE5DE122522
:10308000FF90F0A4E0B1CDE4F5D8E5D820E1FBE570
:10309000DC30E30C90F0A5D1E6B1B944081225ED7F
:1030A00075D808E4F5D8E5D820E1FBE5DE30E55435
:1030B00090F0A531A7900005E5DB1225FF900004F4
:1030C000E5DC1225FF900003B1C29000021225FF3B
:1030D000F1B4E4F5D8E5D820E1FB90F0A531A79054
:1030E0000009E5DB1225FF900008E5DC1225FF90C2
:1030F0000007B1C29000061225FFE9B1B9440412DD
:1031000025ED806EF1D631A7900005EFB1C4900097
:10311000041225FF900003E41225FF900002E41240
:1031200025FF900004F1C92404B1BBF1BE31A79082
:103130000005EF1225BAF1B4E4F5D8E5D820E1FB9B
:10314000F1D631A7900009EFB1C49000081225FF15
:10315000900007E41225FF900006E41225FF90007E
:1031600008F1C92408B1BBF1BE31A7900009EF12E4
:1031700025BAD1F52402B1D3E4F5D8E5D820E1FB96
:1031800090F0A531A7900013E5DD1225FF90001205
:10319000E5DE1225FFD0DED0DDD0DCD0DBD0DAD00A
:1031A000D922917790F0A4E0FBA3E0FAA3E0F92202
:1031B00090F0A4D1B6E4A3F0122574146026147024
:1031C00002414514700241531460552404600241C9
:1031D000C130020B31A4209202807D740241BE31C5
:1031E000A4E441BED1FE400C30920690F046E0606F
:1031F00003309412B1837B017AF0793E51C2D1DF62
:1032000031A4740141B490F046E0FF64016005EF21
:103210006402700631A4740441BE31A4740141BE3D
:1032200090F046E0700431A4802E309412B1837B7C
:10323000017AF0793E51C2D1DF31A4740480753136
:10324000A474048079B183D1D851C2D1BF31A474A0
:1032500003806B20921A31A474011225EDE490F0E2
:1032600034F1E3740AF0B1837B017AF07932805251
:1032700090F046E06401700631A47404804078192F
:103280007CF07D01D1D87E007F081228CBEF3395EA
:10329000E04F600CD1BFD1D851C231A47403801E5D
:1032A000D1FE5016B1837B017AF0793E51C2D1DF55
:1032B00031A474031225ED023FFA31A474031225E0
:1032C000ED2290F0A8D1B678AB7CF07D017BFF7A3F
:1032D000007929D1CBE490F0B3F0A3F0FC90F0A8F2
:1032E000D1E64A4B601390F0A8A3A3E0F9D1D270C5
:1032F0000BD10A7007D10470037F01227B017AF0A1
:10330000792171C790F0A831A7D1D2FF90F026E0C3
:103310002F90F0B0F0E0C3943C74809480400AE0B9
:1033200024C4F090F0B37401F0D10AFF90F024E0CF
:103330002FFF90F0B3E02F90F0AEF0E0C39418743C
:10334000809480400AE024E8F090F0B47401F0D159
:1033500004FF90F023E02FFF90F0B4E02F90F0AD49
:10336000F090F021E024D0FFE43407FEA3E0FD124A
:103370004314AC0790F0ADE0D39C4018E09CF09073
:10338000F023E0FF90F0ADE0B5070990F023E014E2
:1033900090F0ADF0E490F0AFF0A3E0B1B2FD7F09A2
:1033A000917790F0AEE0B1B2FD7F0A917790F0ADE9
:1033B000E0B1B2FD7F0B91777D807F0C91777D022C
:1033C0007F0191777F002290F0B5D1B690F0B5D112
:1033D000E64A4B60707F029146EF547FB16D31A792
:1033E000900006EF1225FF7F039146EF547FB16DE9
:1033F00031A7900005EF1225FF7F04B16831A79037
:103400000003EF1225FF7F05B16831A7900002EF9E
:103410001225FF7F069146EF5407FF90F0B531A7C4
:10342000900004EF1225FF7F079146EF541FB16D06
:1034300031A7900001EF1225FF7F089146B16E3150
:10344000A7EF1225ED22AD07B1947FA2B10BB19485
:103450007FA3B13CB113F10AC204B1DDC205916C86
:1034600000D205B18F0000000000D205E4F5B243A0
:103470008608A205928322AC07B1947FA2B13CB129
:1034800013AF04B10B80D590F0A4D1B6E4A3F0FD46
:1034900090F0A4D1E64A4B605E7F029146EF5480E3
:1034A000FD31A4900006B1AF4DFD7F0231A2900026
:1034B00005B1AFFD7F0331A2D10AD1EEFD7F04310A
:1034C000A2D104D1EEFD7F0531A290000412258D1A
:1034D0005407FD7F0631A2F186FF91F890F0A7E036
:1034E000F1EAEF541F4EFD7F0731A2122574FF91C0
:1034F000F8AD077F08917722EF75F00A84C454F085
:10350000FEEF75F00A84E5F04EFF22B13CB113AF37
:1035100005B13CD205916C0000000000D205B18FCE
:10352000E4F5B25386F70000000000308308C205BE
:10353000B18F915CC322C205B18FD322E4FEF18C1E
:103540005025EF30E704D2058002C205916C0000DF
:10355000000000D205B18FEF25E0FF000000000061
:10356000C205B18F0E80D7229146EF543FFFB17450
:1035700090F0B522EFC4540F75F00AA4FEEF540F7B
:103580002EFF227F019146EF54F7FD7F018177A244
:1035900005928222D205916C00D205B18F00000005
:1035A0000000C205916C0000000000C20580E0121E
:1035B000258DFF91F8EF547F222401F9E43AFA02B5
:1035C0002574E5DD1225FFE5DE541F22EF75F008B6
:1035D000A42407FFE5F03404F5DA8FD9223004047F
:1035E000C2058002D205916C0000000000D205B136
:1035F0008F0000000000C205B18FD205916C000061
:103600000000002290000202258D90000302258D0B
:10361000D1B078A87CF07D017BFF7A007900D1CB16
:1036200090F0A531A712257490F0AAF0F18690F0E1
:10363000ABF0D10490F0A8F0D10A90F0A9F090007E
:103640000412258D90F0AEF0D1D290F0AFF0900042
:103650000612258D90F0ACF090000712258D90F0A9
:10366000ADF090F0A4E0FF123CA190F0A4E0FF7B4D
:10367000017AF079A8123D0390F0A4E0FFE5D8208C
:10368000E1FBC0D9C0DAC0DBC0DCC0DDC0DEB1CC3C
:10369000E4F5DCF5DB75DE0775DD2075D8F1E5D8DE
:1036A00020E1FBD0DED0DDD0DCD0DBD0DAD0D922F7
:1036B00090F0A4EFF0A3EBF0A3EAF0A3E9F02278F6
:1036C000197CF07D017B017AF0794B7E007F080246
:1036D00029BB90000502258D7B017AF0794B22C22F
:1036E00080D296C2B622E0FBA3E0FAA3E022FF91CB
:1036F000F8EF543F2290F0A4E075F008A4227F0177
:103700009146EF5408C36001D322E4F5B25386F723
:10371000FEF18C501FD205B18F0000000000EF2594
:10372000E0FF3083034401FFC205B18F00000000B9
:10373000000E80DD2290F0ACD1B690F0B87401F0AC
:10374000A374F0F0A374AFF07B017AF0F912410892
:10375000EF7002FF227B017AF079AF7D08124051B1
:1037600090F0B7E06F60037F002290F0B831A7F1CE
:1037700086FE122574FDEDFF90F0AC31A7EE8FF0C0
:1037800012268C7F012290000102258DEEC3940841
:103790007480948022AC07E4FBEBF18D5015A803F4
:1037A000EC088003A2E713D8FB5401FAFF123E5540
:1037B0000B80E62275D80875D80875D8082213132F
:1037C000543F1225ED90F0A52212258D5403C433E9
:1037D0003354C0FFE922E5DD54FC1313543FFF903E
:1037E000F0A522F0A3F0A3F0A322C4333333548016
:1037F000FE22E4FDE5D820E1FBC0D9C0DAC0DBC081
:10380000DCC0DDC0DE1235CCE4F5D8E5D820E1FB24
:10381000E5DC5401700EF5DC75DB201133E5D820B2
:10382000E1FB7D01D0DED0DDD0DCD0DBD0DAD0D939
:10383000AF0522F5DEF5DD75D8F122E5D820E1FBF4
:10384000C0D9C0DAC0DBC0DCC0DDC0DE1235CC754B
:10385000DC0075DB08E41133E5D820E1FBD0DED0D5
:10386000DDD0DCD0DBD0DAD0D92278867CF07D01C7
:103870007BFF7A0079087E007F141229BBE490F068
:103880009A1237E31237E31237E3F07F0B7117EF29
:10389000605051F77F0B9101E090F02CF090F09187
:1038A000E090F02BF090F092E090F02AF090F093FE
:1038B000E090F029F090F094E090F030F090F095E6
:1038C000E090F02FF090F096E090F02EF090F097CE
:1038D000E090F02DF07F0B113B7B017AF0792912FB
:1038E00034877F0D7117EF600D51F77F0D122FF2A6
:1038F0007F0D113BD2037F077117EF700221CA5170
:10390000F77F079101E090F00BF090F091E090F0DC
:103910000AF090F092E090F009F090F093E090F0CF
:1039200008F090F094E090F00FF090F095E090F0B7
:103930000EF090F096E090F00DF090F097E090F09F
:103940000CF07F07113B90F018E004F090F00CE0D1
:1039500090F046F090F009E0FFE4FCFDFE780812DC
:1039600026DD90F00851D07D3C51C990F043915E26
:103970007C007D1851E851C790F041122FE6941F4A
:10398000EE940090F0404005741FF08002EFF0903C
:10399000F00BE0FFE4FCFDFE78081226DD90F00A53
:1039A00051D07D3C51C990F050915E7C007D185102
:1039B000E851C790F04E122FE6941FEE940090F05D
:1039C0004D4005741FF08002EFF090F050E090F051
:1039D000E0F090F043E090F0DFF07B017AF0793195
:1039E0001231B030000241A8D2007B017AF0792177
:1039F0001233C7E490F0E4F0A3F090F0E2F0A3F00B
:103A000090F075E0FF90F018E06F704BC20290F0FC
:103A100066E04401F0E04402F090F065E04440F0DC
:103A2000E04480F0A3E04404F0E04410F0E04420DF
:103A3000F0E04408F090F055E04410F03003227BB1
:103A4000017AF079657F0A1236107B017AF0795598
:103A50007F08123610800AD20290F018E090F075BC
:103A6000F0B183A292E433540151FE54FEFDEC7197
:103A70000AA294B3E433540125E0FFE433FE51FF7E
:103A800054FD7107A202E4FE3354017802C333CE21
:103A900033CED8F951FE54FB710730030B7B017A0A
:103AA000F079DE7F0C12361090F054E0FF64406035
:103AB00005EF6480701090F054E090F053F0122BFA
:103AC00069E490F054F0227D18AF03AE0202262183
:103AD000E02FFFE43E90F09EF0A3EFF090F09EE028
:103AE000FAA3E0FB7C007D3CFFAE02122621A3EE90
:103AF000F0A3EFF07C00227B017AF0798622FF9020
:103B0000F0DEE0FCA3E022FDEC4EFEED4FFF90F076
:103B1000DEEEF0A3EFF022E4FDE5D820E1FBC0D912
:103B2000C0DAC0DBC0DCC0DDC0DE1235CCE4F5D8C5
:103B3000E5D820E1FBE5DB30E3027D01D0DED0DD1E
:103B4000D0DCD0DBD0DAD0D9AF05227F057117EFFA
:103B50007002810051F77F059101E090F09DF09097
:103B6000F091E090F09CF090F092E090F09BF0905B
:103B7000F093E090F09AF090F094E090F0A1F09043
:103B8000F095E090F0A0F090F096E090F09FF0902B
:103B9000F097E090F09EF07F05113BC2AFC2C212D9
:103BA0002F7390F09AE064AA700EA3E064AA7008E4
:103BB0007D017F559169813990F09AE064337040BE
:103BC000A3E06433703AF5BFF5BCFD7C03FFFE1241
:103BD0002AFB9108E4FFEFC394207480948050097D
:103BE00074802FF8E4F60F80ED7880761175836F7E
:103BF000E4F5827F80122B2891087D047F5591691E
:103C000022122FF290F09022538FFEE4F5BFFFEFC7
:103C1000C39432748094805020E4FEEE9156501686
:103C2000E4FDED9156500CE5BC30E20453BCFB22A0
:103C30000D80EF0E80E50F80D675BF0175BB9B43ED
:103C40008F0143BB0475BCFF43BB03538FFE75BBA1
:103C5000ABE4F5BF80FEC394FF7480948022EDF046
:103C600090F0A0E0FAA3E0FB2290F0A2EFF0A3ED29
:103C7000F078A47CF07D017BFF7A0079311236CB9D
:103C800090F0A2E090F0A7F090F0A3E090F0A6F002
:103C90007B017AF079A47F09B1037F0912367D7F19
:103CA0000990F0B0EFF0A312271C00000000E47FA1
:103CB000707E17FDFC90F0B1F1EFFBC31226B950F6
:103CC0002A90F0B0E0FF1237F2EF701F12437590A8
:103CD000F0B1E0FCA3F1E72401FFE43EFEE43DFD8A
:103CE000E43CFC90F0B112271080C3223003137F14
:103CF0000691A17B017AF079007F06B1037F06125D
:103D0000367D22E5D820E1FBC0D9C0DAC0DBC0DCBB
:103D1000C0DDC0DE1235CCE4F5DCF5DBF5DE75DDAB
:103D20000875D8F1E5D820E1FB1237B4B16BE5D8BE
:103D300020E1FB75D804740429F9E43AFAB16BE583
:103D4000D820E1FB75D80475D80475DC0075DB401C
:103D500075DE0075DD2075D8F1E5D820E1FBD0DEF9
:103D6000D0DDD0DCD0DBD0DAD0D9221226F0E48E40
:103D7000DC8FDB1226F078101226CA8EDE8FDD75FE
:103D8000D8F122E490F0AAF0A3F01242BCEF700246
:103D9000FF227F647E19D142E490F0A8F0A3F09056
:103DA000F10E122FEB90F0A9E09FEE6480F890F0F6
:103DB000A8E0648098506FE0FCA3E0FD25E0FFECF4
:103DC00033FED129E4F0A3F074D42FF974F03EFA55
:103DD0007B01123735D134D129E0FEA3E0FF124236
:103DE000D090F0A4122710E4FFFE7D207C4190F0DB
:103DF000A4F1EFFB12230F1224F390F0AAEEF0A32C
:103E0000EFF0FDAC06D13474E22FF58274F03EF58C
:103E100083ECF0A3EDF090F0A9E004F0700690F0D0
:103E2000A8E004F0A19F7F012274D42FF58274F0E2
:103E30003EF5832290F0A9E025E0FF90F0A8E03362
:103E4000FE22D3EF9400EE940040090000EF1F70B3
:103E5000011E80EE22AD0712427E7F02FED142AFEC
:103E600005EF3395E0FEEF64014E7002D2B57F1985
:103E70007E00D142D2B57F057E0080C690F08612CA
:103E800036B6E4A3F0788B7CF07D017BFF7A007975
:103E900039FE7F051229BBE490F0D0F0A3F0A3F027
:103EA000124172EF7003FEFF227FF0123795E4900B
:103EB000F08AF090F08AE012378D4002E184E4FA53
:103EC000EA12378D4002E14E12429FEF5403FF90F9
:103ED000F0D0E0FEC313F0EF64027007FFF1B6E428
:103EE000F08068EF64017007F1AD7401F0805CEF61
:103EF0006002E1A990F08AE075F008A42A04FC9021
:103F0000F089E0F9F1D5E0FBECD39B4012E4FFF13E
:103F1000B6E4F090F089E004F0F1D5ECF0802CEC00
:103F2000C39B5013F1B8E0FF54011237EA90F0D070
:103F3000E04EF0D1558014748B29F1D7E06C700BF2
:103F4000F1AD7401F090F089E014F00AC1C090F076
:103F5000D0F1E77803C333CE33CED8F9FF90F086A3
:103F60001236E62FF9EA3EFA90F08AE07E0029F94F
:103F7000EE3AFAED1225EDE490F0D0F090F08AE000
:103F800004F0C1B390F0D2E004F0700690F0D1E0FC
:103F900004F090F089E0F1D5E0600EF1DFC3940504
:103FA000EE648094805002C1A0F1DFFF2290F0D037
:103FB000E04480F07F01D15590F08AE075F008A4CC
:103FC0002AF582E435F0F583E5822490F582E583D5
:103FD00034F0F58322248BF582E434F0F5832290CB
:103FE000F0D1E0FEA3E022E0FDA3E0FEA3E022E0AA
:103FF000F8A3E0F9A3E0FAA3E022C0BF75BF014334
:10400000B40375BB9B43B40475BBABD0BF2290F027
:1040100021E090F003F090F022E090F002F090F0B8
:1040200023E090F001F090F024E090F000F090F0A8
:1040300025E090F007F090F026E090F006F090F088
:1040400027E090F005F090F031E090F004F0023CB1
:10405000EC90F0BB1236B6A3EDF0E4FE90F0BEE0BB
:10406000FD14F0ED6032119B12257490F0BFF0E466
:10407000FFEF12378D50E590F0BFE0FD6E30E00AA3
:10408000EE6418C3134480FE8004EEC313FEEDC338
:104090001390F0BFF00F80D9AF062290F0BBE0FB89
:1040A000A3E475F001122676A9F0FA2290F094129A
:1040B00036B63172EF7002FF227FCC1237957FBE89
:1040C000518711EF90F094119EEF1225ED90F0982A
:1040D000E004F0700690F097E004F0C390F098E0F0
:1040E000940990F097E06480948040D67F0122E4A8
:1040F000FCFBEB12378D500D51778002C333D8FC97
:104100004CFC0B80EDAF042290F0BB1236B6A3ED51
:10411000F03172EF7002FF227F55123795E4F9E912
:1041200012378D502390F0BEE075F008A424E6F518
:1041300082E434F0F583E58229F582E43583F58362
:10414000E0FF1237950980D77FBE123795E490F0D3
:10415000BFF090F0BFE0C3940974809480501011B8
:10416000EF119BEF1225ED90F0BFE004F080E37FAC
:104170000122E4FDFC517F7FF051927F2831ADFB9D
:10418000EB6019C3ED9411EC64809480500E7F05B0
:104190007E0031AEFB0DBD00010C80E47FC87E00C7
:1041A000123E42AF03EB7F0160027F0022FE123E0F
:1041B00042A2B5E43322517E7F0151927F0331AD9B
:1041C000FD7F1B7E00123E42AF052290F094123616
:1041D000B63172EF7002FF227FCC1237957F4E51BD
:1041E0008790F094119E122574FF12379590F098E5
:1041F000E004F0700690F097E004F0C390F098E0CF
:10420000940390F097E06480948040D57F012290E1
:10421000F086EFF0A3EDF090F0917401F0A374F04C
:10422000F0A37488F07B017AF0F911ACEF7002FF13
:10423000227B017AF079887D08115190F090E06F2F
:1042400060037F002290F0911236E624061235BBFF
:1042500054FCFF1225ED90F087E04F1225ED54E35A
:10426000FF1225ED90F086E04F1225ED7B017AF0EC
:10427000798C31CB7F012231B6A803EF0822E4F517
:10428000B243B120C2B522123795E490F097F0A363
:10429000F022FE123E42D2B5E4F5B253B1DF22E481
:1042A000FCFBEBC3940274809480500D5177800224
:1042B000C333D8FC4CFC0B80E9AF04223172EF70A1
:1042C00002FF227FCC1237957F441237957F01225F
:1042D000AD07AC06EC1224BAE4FBFA7980784312FD
:1042E0002418E4FBFA7920784202221EAB07AA06C2
:1042F000EB5403700AFC7D64122621ED4C700FAE66
:1043000002AF037C017D90122621ED4C70037F01EA
:10431000227F002290F0B5EEF0A3EFF0A3EDF0784D
:10432000B87CF07D017BFF7A00791C7E007F0D1246
:1043300029BB90F0B7E0FFC3940174809480400AD9
:10434000D3EF940C7480948040037F002290F0B7E8
:10435000E06402701090F0B5E0FEA3E0FF51ECEFD6
:1043600060037F1D2290F0B7E024B8F582E434F0BA
:10437000F583E0FF22C2AF438F0143BB02538FFEA0
:03438000D2AF2297
:00000001FF
